:020000020000FC
:103C000040C039C030C0415652424F4F54000000AE
:103C10003130000031310000002700936000009334
:103C200061000091600010916100000F111F23E0FE
:103C30006FD10091600010916100000F111F21E110
:103C400067D10091600010E4010F009360000F93B2
:103C5000112700916100011F009361001F91105016
:103C60000E41F8F2089504E00EBF0FE50DBFF89481
:103C70000FEF08BB21C004E00EBF0FE50DBFF894A5
:103C8000CBDFF8940FEF08BB04E00EBF0FE50DBFCC
:103C900011E068D106B305FFBFDFEEEFFBE3C89587
:103CA000002D053A49F4E39509F4F395C895002DE4
:103CB000093E11F40C940000F894EAD0F9D0FED03B
:103CC0000B3111F4F5D0FBCF033739F40EE1FDD001
:103CD00003E9FBD007E0F9D0D9C0033521F4E6E0D1
:103CE000FCE3FCD0D3C0063521F4E0E1FCE3F6D0E0
:103CF000CDC0063721F4E4E1FCE3F0D0C7C00136C3
:103D000019F409E7E2D0C2C0043729F405E7DDD091
:103D100000E0DBD0BBC0043511F4D0D0B5C009370A
:103D200021F4CCD08D9A959AAFC0083721F4C6D033
:103D30008D9A9598A9C0003509F4A6C0003719F4EA
:103D400003E5C3D0A3C00C3409F49EC0053611F4BA
:103D500063DF9AC0033621F4B1D00093620094C0AF
:103D6000033471F4ABD000936300009162001091B2
:103D700063002091600030916100D0D0BCD084C03D
:103D80000D3669F4009160001091610025E0C0D00B
:103D9000009160001091610021E1BAD075C0043437
:103DA000B9F4009160000EBB109161001FBB0F5F62
:103DB0001F4F009360001093610080D00DBB0CB3C7
:103DC00004600CBB02600CBB0CB30270E9F75CC072
:103DD000013459F473D00F9371D01F91000F111F4C
:103DE00010936100009360004FC0023731F401E08E
:103DF000112729E09CD069D049C0063431F400274E
:103E0000112729E094D061D041C0023569F40091B6
:103E100060001091610020E08AD00F93012F55D0EF
:103E20000F9153D068D032C0043691F400916000F5
:103E30000EBB109161001FBB0F5F1F4F009360000E
:103E4000109361000CB301600CBB0DB33ED01EC0DB
:103E50000E3431F403E0112729E069D036D016C0C2
:103E60000C3611F42BD010C0063611F427D00CC03C
:103E7000073411F40C9400000B3119F019D00FE342
:103E800024D016D01CCF08950DE01FD018CF089570
:103E900000E00BB909E109B906D008950F9308E1D4
:103EA0000AB90F9108950F9300E10AB90F9108958F
:103EB0000BB1007811F00CB1FBCF08950BB1007875
:103EC00009F4FCCF0BB10CB10895E8DF0CB90BB1CC
:103ED00000760036E1F7F2DFE6DF0895C895002DA1
:103EE000E39509F4F395C895002A21F00030B1F369
:103EF000ECDFF4CF0895009160001091610022E0A2
:103F0000020F2227121F0093600010936100089592
:103F10001FD0F12FE02F27BFE8951AC019D0F32F3B
:103F2000E22F112E002E21E027BFE89511C010D0FE
:103F3000F12FE02F20FD27BFC895002DE395C895F0
:103F4000102D089505D0002E29E027BFE89500C068
:103F5000022E27B720FDFCCF202D089500000A95E2
:103F6000E9F708950AEFFADF0AEFF8DF0AEFF6DF64
:0A3F70000AEFF4DF1A95B1F7089587
:00000001FF
